:020000040800F2
:100000000000012035270008E5240008E724000847
:10001000E9240008EB240008ED240008000000009B
:10002000000000000000000000000000EF240008B5
:10003000F124000800000000F3240008F524000863
:100040007D2700087D2700087D2700087D27000800
:100050007D2700087D2700087D2700087D270008F0
:100060007D2700087D2700087D2700087D270008E0
:100070007D2700087D270008F924000805250008D1
:10008000112500087D2700087D2700087D2700082E
:100090007D2700087D2700087D2700087D270008B0
:1000A0007D2700087D2700087D2700087D270008A0
:1000B0007D2700087D2700087D2700087D27000890
:1000C0007D2700087D2700087D2700087D27000880
:1000D0007D2700081D250008292500087D27000828
:1000E0007D2700087D2700087D2700087D27000860
:1000F0007D2700087D2700087D2700087D27000850
:100100007D2700087D2700087D2700087D2700083F
:100110007D2700087D270008352500087D27000879
:100120007D2700087D2700087D2700087D2700081F
:1001300000000000000000000000000000000000BF
:1001400000000000000000000000000000000000AF
:10015000000000000000000000000000000000009F
:10016000000000000000000000000000000000008F
:10017000000000000000000000000000000000007F
:10018000000000000000000000000000000000006F
:10019000000000000000000000000000000000005F
:1001A000000000000000000000000000000000004F
:1001B000000000000000000000000000000000003F
:1001C000000000000000000000000000000000002F
:1001D000000000000000000000000000000000001F
:0401E0005FF8E0F1F3
:1001E40010B5054C237833B9044B13B10448AFF36D
:1001F40000800123237010BD800200200000000055
:100204003038000808B5034B1BB103490348AFF36A
:10021400008008BD0000000084020020303800087F
:10022400D0400B1CD1409C46203AD3401843524244
:10023400634693401843704738B50E4B054618780B
:100244004FF47A73B3FBF0F30B4A1068B0FBF3F08E
:1002540000F08CF8044658B90F2D09D802462946F7
:100264004FF0FF3000F042F8044B20461D6038BDCB
:10027400012038BD000000201802002004000020E6
:10028400074A08B51368032043F01003136000F015
:100294001BF80020FFF7D0FF02F00AF8002008BD89
:1002A40000200240034A044B11681B780B4413607E
:1002B400704700BFF802002000000020014B1868BE
:1002C400704700BFF8020020074A0002D36800F418
:1002D400E06023F4E0631B041B0C43F0BF6343F4AE
:1002E40000330343D360704700ED00E0174B30B593
:1002F400DC68C4F30224C4F10703251D042B28BFC2
:100304000423062D4FF0010598BF002405FA03F3DA
:1003140003F1FF3388BF033C1940A14005FA04F4FC
:10032400013C2240002842EA01024FEA0212AFBF18
:1003340000F16040064B00F00F00D2B2A5BFD2B26C
:1003440000F561401A5480F8002330BD00ED00E050
:1003540014ED00E00123420900F01F0003FA00F04D
:10036400014B43F82200704700E100E00138B0F18E
:10037400807F0AD2F021064B064A586082F8231087
:100384000020072298601A6070470120704700BF60
:1003940010E000E000ED00E010B5002832D0016864
:1003A400194B1424994225D8184AA3F207430A4446
:1003B400B2FBF4F2920002648468C36343680A687F
:1003C4002343C46822F47F522343046922F0300299
:1003D40023434469234384692343C4692343134364
:1003E4000B600122002380F82120836380F82030F1
:1003F400184610BD064B0B44B3FBF4F39B00036497
:10040400044BD9E7012010BD07040240F8FFFDBFEB
:10041400F8FBFDBF00040240F0B590F82040012C29
:1004240035D0012490F8215080F82040A5424FF0A7
:1004340000064FF0020428D180F821400468866346
:100444002668076C26F001062660C66BBD40756001
:10045400636043680568102BC36A0BBFA260A16088
:10046400E160E2604BB1236843F00E0323602B6824
:10047400002043F001032B60F0BD236823F0040344
:100484002360236843F00A03F0E780F82060022029
:10049400F0BD000090F8213010B5022B03D00423E6
:1004A4008363012010BD03681A6822F00E021A60EB
:1004B4001A6822F001021A60294A934224D902F5EB
:1004C4006272934219D01432934218D01432934278
:1004D40017D0143293420CBF4FF480534FF480333F
:1004E400204A53600123002480F82130436B80F8B4
:1004F40020409BB39847204610BD0123F0E710230A
:10050400EEE74FF48073EBE717498B4216D01431B2
:100514008B4215D014318B4214D014318B4214D039
:1005240014318B4214D014318B4214D0934214BF33
:100534004FF480334FF080730C4AD2E70123FBE77A
:100544001023F9E74FF48073F6E74FF48053F3E791
:100554004FF48033F0E74FF48013EDE7184610BDF5
:1005640080000240000402400800024000000240F3
:1005740070B40425C66B026C346803689540254248
:10058400196855D04D0753D51A6896065EBF1A6888
:1005940022F004021A60604A93421FD902F5627283
:1005A400934214D01432934213D01432934212D093
:1005B400143293420CBF4FF480434FF48023574AC4
:1005C4005360C36A002B00F0A58070BC1847042355
:1005D400F5E74023F3E74FF48063F0E750498B429B
:1005E40016D014318B4215D014318B4214D01431EF
:1005F4008B4214D014318B4214D014318B4214D05A
:10060400934214BF4FF480234FF08063454AD7E7E9
:100614000423FBE74023F9E74FF48063F6E74FF444
:100624008043F3E74FF48023F0E74FF48003EDE7D2
:1006340002259540254257D08D0755D51A68940652
:1006440006D41A6822F00A021A60012280F82120D6
:10065400314A93421ED902F56272934213D0143286
:10066400934212D01432934211D0143293420CBFED
:100674004FF400534FF40033284A5360002380F8AA
:100684002030836A9EE70223F6E72023F4E74FF441
:100694000073F1E722498B4216D014318B4215D0F6
:1006A40014318B4214D014318B4214D014318B4248
:1006B40014D014318B4214D0934214BF4FF400333E
:1006C4004FF00073174AD8E70223FBE72023F9E72A
:1006D4004FF40073F6E74FF40053F3E74FF400339D
:1006E400F0E74FF40013EDE708259540254211D0BB
:1006F40009070FD5196821F00E011960012303FAC7
:1007040002F27260836380F82130002380F8203085
:10071400036B57E770BC704780000240000402403E
:100724000800024000000240114AD36813F010038D
:1007340005D01049CB6943F00203CB611023D26882
:10074400500706D50B4943F00403CA6942F001027D
:10075400CA61074AD169C90708D50648C16941F089
:100764000401C161D16921F00101D161D3607047F5
:100774000020024000030020064B186910F080009E
:1007840007D0054A5A6002F188325A601869C0F3EA
:10079400C01070470020024023016745034A00202F
:1007A400136943F080031361704700BF00200240C7
:1007B400014BD869704700BF00030020F8B5064616
:1007C400FFF77CFD114C07462546E368D80712D491
:1007D400E368990644BF2023E360EB68DA0606D495
:1007E400EB69DB0703D4E86810F0040002D0FFF7DC
:1007F4009BFF0120F8BD731CE7D00EB90320F8BDA0
:10080400FFF75CFDC01B8642DFD2F7E70020024001
:100814002DE9F84F1F4C9946237E0546012B0F46C0
:10082400904633D001234CF250302376FFF7C6FFB5
:1008340040BB012D03D0022D0CBF02250425002648
:10084400B246DFF854B0320140464946FFF7E8FCAF
:10085400C4F81CA0DBF8103080B243F00103CBF8DD
:10086400103027F816004CF25030FFF7A7FFDBF8E2
:10087400103023F00103CBF8103018B90136F3B26D
:100884009D42E0D800232376BDE8F88F0220BDE81E
:10089400F88F00BF00030020002002400022064B16
:1008A400DA61064B1A6942F004021A611A6942F0CD
:1008B40040021A61704700BF00030020002002407C
:1008C4000022064BDA61064B1A6942F002021A61F1
:1008D40058611A6942F040021A617047000300200F
:1008E400002002402DE9F041234D07462B7E884627
:1008F400012B3DD0012403682C76022B4CF250309E
:1009040013D1FFF75BFF20B1012000232B76BDE854
:10091400F081FFF7C3FF4CF25030FFF74FFF174A47
:10092400136923F004031361EFE7FFF747FF00287F
:10093400EAD14FF0FF33C8F800302046BE680F4CB0
:10094400FA68BB6803EBC2239E42DED23046FFF74F
:10095400B7FF4CF25030FFF731FF236923F0020355
:10096400236110B1C8F80060CFE706F50066E7E739
:100974000220BDE8F08100BF0003002000200240F7
:100984002DE9F74F002216466C4F6D4BDFF8B8E1A6
:10099400DFF8B8C14FF001080C6808FA06F808EA55
:1009A4000404A04540F085804D68122D00F0B78006
:1009B40000F28D80022D00F0AF8000F28180002DC6
:1009C40000F09180012D00F0A5804FF00F09FF2C5D
:1009D40093BF824606F18045083DD0F800B092BF2F
:1009E400B500D0F804B0AD0009FA05F82BEA080800
:1009F40002FA05F588BF00F1040A48EA0505CAF8B9
:100A04000050D1F804A01AF0805F52D0BD6926F0DE
:100A1400030845F00105BD61BD6908F1804805F092
:100A24000105019508F5803806F0030B019D4FEA96
:100A34008B0BD8F8085009FA0BF925EA0909414D3E
:100A4400A84271D005F58065A8426FD005F5806590
:100A5400A8426DD005F58065A8426BD005F5806588
:100A6400A84269D070450CBF0525062505FA0BF58B
:100A740045EA0905C8F808501D681AF4803F14BFF8
:100A84002543A5431D605D681AF4003F14BF254348
:100A9400A5435D609D681AF4801F14BF2543A543D8
:100AA4009D60DD681AF4001F14BF2C4325EA04047A
:100AB400DC600136102E7FF46DAF03B0BDE8F08F1B
:100AC400032D25D0112D80D1CA6804327DE76545F8
:100AD40009D012D8DFF878904D4504D009F5803953
:100AE4004D457FF472AF8A68E2B1012A0CBFC0F8A9
:100AF4001080C0F81480082267E7DFF858904D454D
:100B0400F1D009F580394D45EDD0A9F58019E7E715
:100B140000225AE7CA6858E7CA68083255E7CA6823
:100B24000C3252E7042250E700259FE701259DE798
:100B340002259BE7032599E7042597E70010024067
:100B44000004014000080140001C01400000211085
:100B540000001110000031100AB10161704709044E
:100B6400FBE7C3685940C1607047000038B50446CC
:100B740008B9012038BD90F83D3003F0FF021BB9DD
:100B840080F83C2001F0B6FB2423226884F83D3031
:100B9400136823F00103136000F0E2FA63682F4A3C
:100BA400934230D82E4A9042E3D92E4A2168B0FBB2
:100BB400F2F24A6001320A62284A0138934232D87A
:100BC4005B00B0FBF3F0431CC3F30B03042B38BFEF
:100BD4000423CB61226AE369002013430B60E268BB
:100BE400236913438B60A26963691343CB600B6869
:100BF40043F001030B602023206484F83D3020631C
:100C040084F83E0038BD184A9042B2D9154D4FF4CD
:100C14009672B0FBF5F521686A434D604FF47A751E
:100C2400B2FBF5F2C6E7A26852B903EB4303B0FB8B
:100C3400F3F0431CC3F30B036BB143F40043C8E765
:100C440019225343B0FBF3F0431CC3F30B0313B15A
:100C540043F44043BDE70123BBE700BFA086010086
:100C64007F841E0040420F00FF083D0003682DE909
:100C7400F341DB07054610D42B689F075ED42B682D
:100C8400190700F195802B685A0700F1BF80EA69C3
:100C9400002A40F02D81002014E0904C636803F09A
:100CA4000C03042B07D0636803F00C03082B0CD14E
:100CB4006368DE0309D523689C03DDD56B68002BCC
:100CC400DAD1012002B0BDE8F0816B68B3F5803F52
:100CD40010D1236843F480332360FFF7EFFA06460C
:100CE40023689803C8D4FFF7E9FA801B6428F7D96E
:100CF4000320E7E79BB9236823F480332360236848
:100D040023F480232360FFF7D9FA06462368990366
:100D1400B2D5FFF7D3FA801B6428F7D9E8E7B3F517
:100D2400A02F236803D143F480232360D1E723F465
:100D340080332360236823F48023CDE7674C636802
:100D440013F00C0F07D0636803F00C03082B10D1C9
:100D54006368DA030DD423689B0702D52B69012B42
:100D6400AFD123686A6923F0F80343EAC20323601E
:100D740085E72A695A4B6AB101221A60FFF79EFA85
:100D8400064623689F07ECD4FFF798FA801B0228D5
:100D9400F7D9ADE71A60FFF791FA0646236898077A
:100DA4007FF56DAFFFF78AFA801B0228F6D99FE71B
:100DB400AA694A4C4B4BDAB101221A60FFF77EFA5A
:100DC4000646636A9B070DD54FF4FA52464B1B68DF
:100DD400B3FBF2F3019300BF019B5A1E0192002B57
:100DE400F9D150E7FFF76AFA801B0228E9D97FE7B7
:100DF4001A60FFF763FA0646636A9F077FF543AFFD
:100E0400FFF75CFA801B0228F6D971E7334CE369DB
:100E1400D80024D40127E36943F08053E361E369F4
:100E240003F080530093009B304E3368D90518D5E6
:100E3400EB68012B26D1236A43F001032362FFF7F9
:100E44003DFA41F288368046236A9B073FD5002F3E
:100E54003FF41DAFE36923F08053E36117E70027F4
:100E6400E2E7336843F480733360FFF727FA804680
:100E74003368DA05DCD4FFF721FAA0EB0800642814
:100E8400F6D935E7ABB9236A41F2883823F0010378
:100E94002362236A23F004032362FFF70FFA064652
:100EA400236A9807D3D5FFF709FA801B4045F7D981
:100EB4001EE7052B236A03D143F004032362BAE738
:100EC40023F001032362236A23F00403B6E7FFF748
:100ED400F5F9A0EB0800B042B6D909E700100240CA
:100EE4000000424280044242180200200070004088
:100EF400224C636803F00C03082B3FF4E2AE00239A
:100F04001F4E022A33602BD1FFF7D8F90746236816
:100F140099011FD42B6AB3F5803F05D16268A96893
:100F240022F400320A436260696A62680B4322F465
:100F340074121343636001233360FFF7BFF905465E
:100F440023689A013FF5A7AEFFF7B8F9401B0228C2
:100F5400F6D9CDE6FFF7B2F9C01B0228D7D9C7E608
:100F6400FFF7ACF9054623689B017FF594AEFFF7C4
:100F7400A5F9401B0228F6D9BAE600BF00100240CA
:100F84006000424230B5194B87B002AC03F1100542
:100F9400224618685968083303C2AB421446F7D195
:100FA40001238DF80430022311498DF805304B6874
:100FB40003F00C02082A17D1C3F3834206A80244A3
:100FC400DB0312F8102C0CD54B680A48C3F34043DA
:100FD400504306AA134413F8143CB0FBF3F007B0D3
:100FE40030BD05485043FAE70248F8E7483800089E
:100FF4000010024000127A0000093D00544A2DE915
:10100400F0411368054603F007038B420E462AD3CA
:1010140029688C0734D4CA0747D44D4A136803F0AF
:1010240007039E42C0F082802A684A4C12F0040FE3
:1010340040F08780130706D563682A6923F4605358
:1010440043EAC2036360FFF79DFF6368424AC3F348
:101054000313D35CD840414B18600020FFF7ECF831
:101064000020BDE8F081136823F007030B431360ED
:10107400136803F007039942CAD00120BDE8F08148
:10108400344B11F0040F1EBF5A6842F4E0625A60F8
:10109400080742BF5A6842F460525A605A68A86806
:1010A40022F0F00202435A60B5E76A68294C012A2B
:1010B40023681CD113F4003FDFD0636841F2883801
:1010C40023F0030313436360FFF7F8F86B680746E4
:1010D400012B14D1636803F00C03042B9DD0FFF79C
:1010E400EDF8C01B4045F5D90320BDE8F081022A84
:1010F40002D113F0007FDFE713F0020FDCE7022BCD
:101104000FD1636803F00C03082B86D0FFF7D6F8E1
:10111400C01B4045F5D9E7E7FFF7D0F8C01B4045B1
:10112400E2D8636813F00C0FF6D176E7136823F066
:10113400070333431360136803F007039E429CD1F3
:1011440072E76368E96823F4E0630B43636071E763
:1011540000200240001002405A3900081802002002
:10116400044B054A5B68C3F30223D35C034A10684B
:10117400D8407047001002406A3900081802002065
:10118400044B054A5B68C3F3C223D35C034A10686B
:10119400D8407047001002406A3900081802002045
:1011A40003680020DA6842F00102DA601A6842F04B
:1011B40001021A60704770477047704770470368B0
:1011C40010B51A69044691070ED5DA6892070BD553
:1011D4006FF002021A6101229B6902779B0777D0A4
:1011E400FFF7EAFF0023237723681A69500710D515
:1011F400DA6851070DD56FF004021A6102229B6967
:10120400227713F4407F204668D0FFF7D5FF0023F0
:10121400237723681A6912070FD5DA6810070CD5EB
:101224006FF008021A610422DB69227799072046CD
:101234005AD0FFF7C1FF0023237723681A69D20627
:1012440010D5DA68D0060DD56FF010021A610822A5
:10125400DB69227713F4407F20464BD0FFF7ACFFC5
:101264000023237723681A69D10708D5DA68D207DF
:1012740005D56FF0010220461A6100F0C5FE23680F
:101284001A69100608D5DA68110605D56FF08002D0
:1012940020461A6100F0BFF823681A69520608D57F
:1012A400DA68500605D56FF0400220461A61FFF750
:1012B40085FF23681A69910622D5DA6892061FD53C
:1012C4006FF020022046BDE810401A6100F0A2B879
:1012D400FFF771FF2046FFF770FF83E7FFF76BFF0F
:1012E4002046FFF76AFF92E7FFF765FF2046FFF706
:1012F40064FFA0E7FFF75FFF2046FFF75EFFAFE75D
:1013040010BD0000244A0368904212D002F5006226
:1013140090420ED0B0F1804F0BD0A2F5983290429B
:1013240007D002F58062904203D002F580629042B9
:101334001DD14A6823F070031343174A904212D018
:1013440002F5006290420ED0B0F1804F0BD0A2F5AE
:101354009832904207D002F58062904203D002F5A1
:101364008062904203D1CA6823F4407313434A69EC
:1013740023F08003134303608B68C3620B688362AA
:10138400054B984203D003F50063984201D10B69E1
:101394000363012343617047002C014010B50446E8
:1013A400A0B190F83D3003F0FF021BB980F83C2057
:1013B40000F0D2FF0223206884F83D30211DFFF79E
:1013C400A1FF0123002084F83D3010BD012010BD91
:1013D40090F83C3010B5012B4FF0020318D080F880
:1013E4003D3003680C685A68496822F070025A60FC
:1013F4005A6822435A609A6822F080029A609A6876
:101404000A439A60012380F83D30002380F83C3081
:10141400184610BD704770470368DA6822F490726A
:10142400DA605A6922F001025A61202380F83A30C6
:10143400704700002DE9F0470568C2682B6901690F
:1014440023F4405313432B618368EA680B434169D7
:1014540022F4B05222F00C020B431343EB606B698D
:10146400826923F4407313436B61404B81469D4270
:101474004FF0190446D1FFF783FE04FB00F3D9F8BB
:1014840004604FF06408B600B3FBF6F3B3FBF8F363
:101494001E01FFF775FE6043D9F804309B00B0FBD2
:1014A400F3F7FFF76DFE6043D9F804309B00B0FBFF
:1014B400F3F3B3FBF8F308FB13731B013233B3FBF1
:1014C400F8F303F0F007FFF75BFE6043D9F804205C
:1014D4009200B0FBF2FAFFF753FE6043D9F80430F0
:1014E4009B00B0FBF3F3B3FBF8F308FB13A31B015E
:1014F4003233B3FBF8F303F00F033B433344AB60E5
:10150400BDE8F087FFF72CFE04FB00F3D9F8046074
:101514004FF06408B600B3FBF6F3B3FBF8F31E0117
:10152400FFF71EFE6043D9F804309B00B0FBF3F7CD
:10153400FFF716FE6043D9F804309B00B0FBF3F3C9
:10154400B3FBF8F308FB13731B013233B3FBF8F35B
:1015540003F0F007FFF704FE6043D9F8042092007B
:10156400B0FBF2FAFFF7FCFDB7E700BF003801401B
:10157400F8B504460E4617461D4621680B6836EA40
:10158400030301D10020F8BD6B1CF7D095B9236883
:101594000320DA6822F4D072DA605A6922F0010278
:1015A4005A61202384F8393084F83A30002384F8CF
:1015B4003830F8BDFEF782FEC01B8542DDD2E6E777
:1015C40010B5044640B390F8393003F0FF021BB95C
:1015D40080F8382000F0D4FE2423226884F83930BF
:1015E400D368204623F40053D360FFF723FF236816
:1015F40000201A6922F490421A615A6922F02A02E0
:101604005A61DA6842F40052DA602023E06384F815
:10161400393084F83A3010BD012010BD2DE9F04175
:101624001F4690F839300446202B0D4690464ED183
:10163400002949D0002A47D090F83830012B46D0F1
:10164400012380F838300023C363212380F8393024
:10165400FEF734FE0646A4F82480A4F82680E38C22
:101664009BB26BB93B46324640212046FFF780FFD0
:10167400A8B9202384F8380084F83930BDE8F08113
:10168400E38C3246013B9BB2E384A3688021B3F52B
:10169400805F20463B460ED1FFF76AFF10B103205E
:1016A400BDE8F0812B882268C3F3080353602369E3
:1016B40043B90235D3E7FFF75BFF0028EFD1236876
:1016C4002A785A600135CAE70120BDE8F08102207A
:1016D400BDE8F081134690F83A2073B5202A0546F8
:1016E40038D1002934D0002B32D090F83820012A88
:1016F40030D00122002480F83820222281628385A0
:10170400C46380F83A20406B134A2E688262134AFD
:101714004463C262124A02630A46311DFEF77CFE2C
:1017240020462B6801941A6801925A6885F838405B
:101734000192019ADA6842F48072DA605A6942F0DE
:1017440001025A615A6942F040025A6102B070BD06
:101754000120FBE70220F9E76B17000821180008B5
:101764002D180008704708B50368426A1B6813F017
:10177400200310D1D3851368D96821F48071D9600E
:10178400596921F001015961596921F040015961F8
:10179400202382F83A30104600F09AFF08BD90F8F2
:1017A4003A3010B5222B36D183680169B3F5805FD6
:1017B4000268836A23D15268E9B9C2F3080223F8A4
:1017C400022B8362C48D013CA4B2C4858CB9036826
:1017D400DA6822F02002DA60DA6822F48072DA60D1
:1017E4005A6922F001025A61202380F83A3000F04D
:1017F4006FFF002010BDD2B223F8012BE1E721B91D
:10180400591C526881621A70DCE75268591C816263
:1018140002F07F02F7E7022010BD704708B5406A66
:10182400FFF7FBFF08BD7047416A08B50B685A69AA
:1018340091F8390021280AD1120608D50022CA8459
:10184400DA6822F0C002DA60202281F839205B696C
:1018540091F83A20222A06D15B0604D500230846D3
:10186400CB85FFF7D9FDCB6B084643F01003CB6360
:10187400FFF7D9FF08BD0000036870B51A68044675
:101884001607D9685D6907D196065AD58D0658D5CD
:10189400BDE87040FFF783BF15F0010502D111F4D4
:1018A400907F4ED0D30705D5CE0542BFE36B43F0FE
:1018B4000103E363500704D51DB1E36B43F0020356
:1018C400E363930704D51DB1E36B43F00403E363BF
:1018D400160704D51DB1E36B43F00803E363E36B20
:1018E400002B66D0950604D5880602D52046FFF75E
:1018F40056FF236820465D69E26B110702D415F098
:1019040040051AD0FFF788FD23685A69520610D59E
:101914005A69606B22F040025A6150B1254B43630F
:10192400FEF7B8FD002844D0606BBDE87040436BFF
:1019340018472046FFF777FF70BDFFF774FFE56394
:1019440070BD160627D50D0625D594F83920212A11
:101954002FD1A268B2F5805F226A17D11188C1F332
:1019640008015960216979B902322262E28C013A94
:1019740092B2E284EAB9DA6822F08002DA60DA68C4
:1019840042F04002DA6070BD0132EEE7511C216280
:1019940012785A60EAE750060BD54A0609D5DA6888
:1019A400204622F04002DA60202384F83930FFF721
:1019B400D9FE70BDBD19000808B50023406AC3856F
:1019C400C384FFF730FF08BD10B5064CA178601C36
:1019D40000F0BEF8A178207103312046BDE8104024
:1019E40000F09CBE0E00002070B5817804464318B8
:1019F4005A78013000F0C7F801280ED000231E4E9B
:101A0400A2785D1C0232DBB29A422DDA1B4800F048
:101A14005BFF22221A4B5A700EE01122184D6A7095
:101A24006278DD2A01D0EE2A06D1204600F06EFA53
:101A3400012801D122236B70114DA978681C00F094
:101A440087F828716378EE2B06D00A2B04D0A97886
:101A54002846033100F062FE6378EE2B0AD1BDE81C
:101A64007040084800F030BFE15C304600F0B8FE3A
:101A74002B46C5E770BD00BF583800085E38000823
:101A8400080000206F380008002310B5C11C143072
:101A940011F8014F23448142DBB2F9D19B1A584219
:101AA400584110BDC21C00F11403002012F8011F9C
:101AB40008449A42C0B2F9D170470000002310B51F
:101AC4000F4CC90007290FDC61B141F2210213F464
:101AD400004F4FEA43039BB201F1FF3118BF53405B
:101AE4000029F4D1184610BD10F8012B083982EAF8
:101AF400132234F8122082EA03239BB2E2E700BFE8
:101B040014000020002330B5104DC900072911DC52
:101B140061B141F2210013F4004F4FEA43039BB239
:101B240001F1FF3118BF43400029F4D1981A18BFBE
:101B3400012030BD10F8014B083984EA132435F82C
:101B4400144084EA03239BB2E0E700BF14000020A2
:101B540010B5FF230446221AD2B2914201D8184686
:101B640010BD14F8012B5340082213F0800F02F12A
:101B7400FF324FEA430318BF83F0310312F0FF0230
:101B8400DBB2F2D1E7E730B5FF2305462C1AE4B205
:101B9400A14203D89B1A5842584130BD15F8014B55
:101BA4006340082413F0800F04F1FF344FEA430329
:101BB40018BF83F0310314F0FF04DBB2F2D1E5E780
:101BC4002DE9F04101F1200323F0070300AFADEB51
:101BD400030D04460E46FFF771FF0DEB0603020AE0
:101BE4009A750322D8751A7616238DF800308DF86D
:101BF40001308DF802308DF80330F12300258DF883
:101C04000530A37968468DF80630E3798DF80450E1
:101C14008DF80730237A8DF811508DF80830637AE7
:101C2400E8468DF80930A37A8DF80A30E37A8DF806
:101C34000B30237B8DF80C30637B8DF80D30A37B48
:101C44008DF80E30E37B8DF80F30237C8DF8103047
:101C5400330A8DF813308DF81460FFF723FF2B46F9
:101C64008DF81500122B1CBF18F80320E254013321
:101C7400162BF7D100230133042B03D12046BD4694
:101C8400BDE8F0819A19A1184244527D4A75F2E7E1
:101C94002DE9F843837C0446103B042B00F28D802D
:101CA400DFE803F0031949717E000323C3760023A0
:101CB400037743778377C37780F8203080F8213027
:101CC4009023A3740C212046FFF77AFFBDE8F84364
:101CD400252100F023BDC37E827E1B0403EB026337
:101CE400427F374E1344027F074603EB02233360DF
:101CF40000231D46DFF8D880DFF8D8908377C377B8
:101D040080F8203007F8213F3368D8F800209B1A68
:101D14009D4209D92B49204600F022F9336801334A
:101D2400C8F800309123CCE717F8011F484600F0AB
:101D340057FD0135E8E7C57D837D2D0445EA03653C
:101D4400437E1F4E1D43037E316845EA03258D42C1
:101D540003D02A461C4800F043FDA27EE37E03EB39
:101D640002239BB223B12A463168184800F038FD9B
:101D7400002323776377A377E37784F8203084F80C
:101D8400213092239DE70323C3760023037743770F
:101D94008377C37780F8203080F82130932390E74D
:101DA4000323C3760023037743778377C37780F8CD
:101DB400203080F82130942383E7BDE8F88300BF06
:101DC4009C0200200050000880380008B038000849
:101DD400A002002058380008B0B50D4A00AFD369FE
:101DE4000C4823F01003D36100F06EFD0A4B0B4A3C
:101DF4001B680B4C0B481360236000F065FD0A4B15
:101E04001B6883F308882368BD46BDE8B0401847C3
:101E1400001002404239000804500008200300204A
:101E24002403002054390008005000082DE9F04133
:101E34000546044600270F4EDFF83C80AB78621B52
:101E4400023B934202DC3846BDE8F0812379E27814
:101E5400316802EB032292B200230120FEF7D8FC82
:101E640018B1404600F030FD0127336802340233D4
:101E74003360E3E714020020273900082DE9F84312
:101E8400044605460027C37E827E1B0403EB0263DF
:101E9400427F1A4E1344027FDFF8688003EB02236B
:101EA400DFF8649033603368D8F80020291B9A1A4D
:101EB400914205D90133C8F800303846BDE8F883AB
:101EC40095F8233095F82220D9F8001002EB03226C
:101ED40092B200230120FEF79BFC30B167B1FEF7FC
:101EE40067FC0146064800F07BFCD9F80030023557
:101EF4000233C9F80030D6E70127F6E7A402002030
:101F0400DF380008D0020020D402002038B50023B6
:101F14000E4C054623600E4BA3601F23E360FEF7BF
:101F24002BFC0C4B1A784AB901220B4920461A7033
:101F3400FEF7D8FC10B1094800F0C6FC2846FFF7AC
:101F440075FF0446FEF72AFC204638BDA80200208F
:101F540000500008D8020020C802002033390008CD
:101F640038B50C460546FEF707FC1C490A78A2B9A9
:101F74001B4B9C421B4B28D017D81B4884421FD0B4
:101F840001220A709A68194B194916481A60FEF71B
:101F9400A9FC10B1174800F097FC2846FFF76EFF24
:101FA4000446FEF7FBFB204638BD1348844210D09C
:101FB40000F580308442E3D11A609C600F4A02E04D
:101FC4001A601F229C60DA60DAE71A609C600C4A8F
:101FD400F9E71A609C600B4AF5E700BFD8020020BD
:101FE40000500108B802002000500008D40200206C
:101FF400CC0200203339000800500208BFFF1F0044
:10200400FFFF1F00DFFF1F000268084B9A420BD13D
:10201400074A136801331360064A136801331360D7
:10202400054A136801331360704700BF0010004075
:10203400E4020020E0020020DC02002010B5144677
:102044000A230248FFF7EAFA204610BD480400209C
:1020540010B590B02822002106A800F0B9FB142284
:10206400002101A800F0B4FB01230A9310230224E9
:102074000B934FF4401306A80F9306940D94FEF7A8
:10208400F5FD0F234FF4806201930023214601A83C
:102094000294039304920593FEF7B0FF10B010BDB1
:1020A40080B588B0FEF7ECF8FFF7D2FF10226F4D31
:1020B40000210DEB020000F08BFBAB69002243F022
:1020C4001003AB61AB694FF4004103F010030193BB
:1020D400019BAB69664843F00403AB61AB69002420
:1020E40003F004030293029BAB690C2643F008033C
:1020F400AB61AB694FF4E13703F008030393039B2F
:10210400FEF72AFD4FF400430493012305930223B1
:1021140004A9574807930694FEF732FC6B695548A7
:1021240043F001036B616B69466103F001030093A3
:10213400009B514B846080E88800C4600461846122
:10214400C461FFF73DFA4D484D4A4E4B846080E828
:102154000C004FF48043C460036144618461C46132
:102164000462FEF703FD41F2DF53474D4749284619
:1021740085E80A000923AC60EB60AC610494059423
:10218400FFF70CF904A9284604940594FFF720F9F5
:102194003F4B404880E8880046618460C460046125
:1021A4008461C461FFF70CFA224621460F20FEF732
:1021B4009DF80F20FEF7CEF8224621462520FEF793
:1021C40095F82520FEF7C6F8224621463620FEF76C
:1021D4008DF83620FEF7BEF8224621460E20FEF783
:1021E40085F80E20FEF7B6F8224621461020FEF7A9
:1021F4007DF81020FEF7AEF8224621462620FEF791
:1022040075F82620FEF7A6F82846FEF7C9FF224BEC
:1022140021461B68164E986800F05EFBFFF7D4FB5E
:102224001E4800F0E5F91E4D1E4C2368B3F5FA7FF5
:1022340006D94FF400413046FEF793FC0023236097
:10224400164C0C4FA368002B02DD2B681E2B03D801
:10225400154F40F6B83405E0384600F0D7F9F1E7F9
:10226400FFF7BAFD3B68A342FAD8DDE7001002404D
:102274000010014048040020003801406C03002095
:1022840000580040801A0600880400200010004016
:1022940000440040C80400201C020020080500205F
:1022A400E4020020E0020020DC020020704700006D
:1022B4000E4B82B09A6942F001029A619A6902F067
:1022C40001020092009ADA6942F08052DA61DB6915
:1022D400074A03F080530193019B536823F0E063A2
:1022E40043F00073536002B0704700BF0010024017
:1022F4000000014010B5044686B01022002102A857
:1023040000F066FA2268114B9A421DD1104C02A9C2
:10231400A369104843F00803A361A36903F0080309
:102324000093009B4FF4406302931223039303230F
:102334000593FEF725FBE36943F48003E361E36956
:1023440003F480030193019B06B010BD00580040C4
:1023540000100240000C01400268084B82B09A420F
:102364000AD103F50033DA6942F01002DA61DB695D
:1023740003F010030193019B02B07047001000406A
:10238400102270B5064688B00DEB0200002100F063
:102394001FFA3368484A934252D1484B04A99A69B8
:1023A400474842F480429A619A69002502F48042C7
:1023B4000092009A9A69434C42F004029A619B6924
:1023C40003F004030193019B4FF40073049302236D
:1023D400059303230793FEF7D3FA4FF48063384839
:1023E40004A9049305950695FEF7CAFA364B2046D0
:1023F40084E828008023A560E36025616561A56108
:10240400E561FDF7C9FF08B1FFF750FF4FF0100C6D
:102414002E4B746366622E4C802284E808100023DD
:102424002046A360E26023616361A361E361FDF779
:10243400B3FF08B1FFF73AFF3463666208B070BDBA
:10244400244A9342FAD11D4B04A9DA691C4842F488
:102454000032DA61DA69002502F400320292029A4B
:102464009A691D4C42F004029A619B6903F00403CB
:102474000393039B042304930223059303230793E9
:10248400FEF77EFA08230E4804A9049305950695E1
:10249400FEF776FA114B204684E828008023A560D5
:1024A400E36025616561A561E561FDF775FF08B12C
:1024B400FFF7FCFE7463C0E70038014000100240DF
:1024C4000008014004040020580002404400024077
:1024D400C003002000440040280300206C00024098
:1024E4007047FEE7FEE7FEE7FEE770477047704778
:1024F400FDF7D8BE0148FEF73BB800BFC00300207B
:102504000148FEF735B800BF040400200148FEF777
:102514002FB800BF280300200148FFF7ADB900BF62
:10252400480400200148FFF7A7B900BFC8040020F1
:102534000148FEF744BE00BF8804002070B50E4673
:1025440015460C46A31B9D4201DC284670BDAFF323
:10255400008004F8010BF5E708B50A4B0246196838
:1025640009B9094919606946186802448A4206D9BA
:1025740000F004F90C2303604FF0FF3008BD1A602B
:1025840008BD00BFE8020020081200204FF0FF3011
:1025940070474FF4005300204B6070470120704790
:1025A400002070470F4B1A6842F001021A60596804
:1025B4000D4A0A405A601A6822F0847222F480326A
:1025C4001A601A6822F480221A605A6822F4FE0201
:1025D4005A604FF41F029A604FF00062034B9A60F6
:1025E400704700BF001002400000FFF800ED00E05B
:1025F4000023012243600360836002490248FFF71D
:1026040069B800BF1405002048040020294A70B5A9
:102614001068294C431C1360284B596803F10C05BE
:102624004D5D0131255440F24B408142C8BF002129
:102634009D685960013D9D607DB923781560BE2B6E
:102644000CD11D48FFF7D0F9002340F24C426355EA
:1026540001359542FBD11A4A136070BD162BF3D194
:102664006378162BF0D1A378162BEDD1E378162BD3
:10267400EAD1627D12211048FFF706FAB0B1E37C7B
:10268400217D104841EA03216318DA7D1E7E46EA63
:1026940002263246FFF736FA18B10748FFF7F8FA70
:1026A400D2E73146084800F09BF8CDE7617D074842
:1026B400F9E700BFEC0200206009002008050020B3
:1026C400DC020020760900207239000880390008F5
:1026D40000220E4B10B51A6040F24B420C4C23689A
:1026E40001339342C8BF00232360A368013393429C
:1026F400A36001DDFFF78AFF236806490122BDE8D4
:10270400104019440448FEF7E5BF00BFE40200206E
:102714000805002014050020480400200A464FF64E
:10272400FF7301460148FEF779BF00BF480400204B
:10273400002103E00B4B5B58435004310A480B4B18
:1027440042189A42F6D30A4A02E0002342F8043BB4
:10275400084B9A42F9D3FFF725FF00F015F8FFF76D
:102764009FFC7047343A00080000002080020020DB
:102774008002002008120020FEE70000014B1868C8
:10278400704700BF1C02002070B500250C4E0D4C94
:10279400A41BA410A54209D101F048F800250A4E53
:1027A4000A4CA41BA410A54205D170BD56F82530CF
:1027B40098470135EEE756F8253098470135F2E79A
:1027C4002C3A00082C3A00082C3A0008303A000849
:1027D40003460244934200D1704703F8011BF9E712
:1027E4000FB40A4B13B51C6824B1A36913B920466E
:1027F40000F0DAFA05AB049AA1682046019300F0D0
:102804009BFC02B0BDE8104004B070471C020020DD
:1028140070B50E46054618B183690BB900F0C4FAC9
:10282400AB69AC6813B9284600F0BEFA234B9C424E
:1028340017D16C68A3891B071DD52369DBB1013E41
:10284400A36816F8011F013BA360E9B9002B2EDA37
:1028540022460A21284600F0F5F8013011D00A205A
:1028640070BD174B9C4201D1AC68E3E7154B9C4209
:1028740008BFEC68DEE72146284600F035F9002859
:10288400DDD04FF0FF3070BD002B04DAA269934213
:1028940006DB0A2904D023685A1C22601970CFE78A
:1028A4002246284600F0CEF80130C9D1E9E70A20D3
:1028B40023685A1C2260187070BD00BFB839000824
:1028C400D839000898390008024B01461868FFF708
:1028D4009FBF00BF1C02002000294FF480630CBF7F
:1028E4000222002200F000B82DE9F7431D46514BA7
:1028F40004461E680F46904626B1B36913B93046A4
:1029040000F052FA4C4B9C4252D17468B8F1020F59
:1029140006D0B8F1010F00F28980002DC0F2868044
:102924002146304600F0D6F9616B41B104F144030D
:10293400994202D0304600F02DFB0023636300234C
:10294400A3616360A3891B0603D52169304600F0A7
:1029540021FBA389B8F1020F23F44A6323F0030394
:10296400A3815DD001AB6A462146304600F0A6FA49
:10297400A3891843A0812DBB009D284600F002FBCB
:10298400074600284ED1DDF80090A9453CD14FF010
:10299400FF30A38943F00203A3810023A36004F161
:1029A4004703236023610123636103B0BDE8F0831F
:1029B400224B9C4201D1B468A8E7214B9C4208BF3A
:1029C400F468A3E7002FD8D0B36913B9304600F0F8
:1029D400EBF9B8F1010F08BFA389276004BF43F0E6
:1029E4000103A381A389276113F0080065611BD04B
:1029F40013F001004FF000031FBF6D42A360A561F7
:102A0400184608BFA560D0E7484600F0BBFA074661
:102A14000028BCD0A3894D4643F08003A381D3E7AB
:102A24000020B6E7A946F5E7A060BEE74FF0FF3007
:102A3400BBE700BF1C020020B8390008D8390008E1
:102A440098390008F8B50E461446054618B183694E
:102A54000BB900F0A9F9214B9C422AD16C68A369F7
:102A6400A360A3891A072ED5236963B32369206859
:102A7400F6B2C01A63693746984204DB21462846F9
:102A840000F028F928BBA3680130013BA360236848
:102A94005A1C22601E706369984204D0A389DB0724
:102AA40019D50A2E17D12146284600F013F990B102
:102AB4000FE00B4B9C4201D1AC68D0E7094B9C4220
:102AC40008BFEC68CBE72146284600F00DF8002843
:102AD400CCD04FF0FF373846F8BD00BFB8390008F6
:102AE400D839000898390008324B70B51D6806467D
:102AF4000C4625B1AB6913B9284600F055F92E4BA5
:102B04009C420FD16C68B4F90C309AB215072CD4DE
:102B1400D00611D40922326043F04003A3814FF060
:102B2400FF3070BD254B9C4201D1AC68EBE7244BD0
:102B34009C4208BFEC68E6E7510712D5616B41B1CE
:102B440004F14403994202D0304600F023FA0023F2
:102B54006363A38923F02403A381002363602369AF
:102B64002360A38943F00803A38123694BB9A38994
:102B740003F42073B3F5007F03D02146304600F000
:102B8400C1F9A28912F001030CD00023A360636988
:102B94005B42A361236953B9B4F90C3013F080008C
:102BA400BAD170BD920758BF6369A360F2E70020F1
:102BB400F7E700BF1C020020B8390008D839000824
:102BC400983900088A892DE9F041054610070C461A
:102BD4005AD44B68002B05DC0B6C002B02DC002064
:102BE400BDE8F081E66A002EF9D0002312F4805289
:102BF4002F682B6033D0606DA3895A0705D56368AD
:102C0400C01A636B0BB1236CC01A00230246E66A38
:102C1400216A2846B047431CA38906D129681D2987
:102C24004BD82B4ACA40D60747D500226260226996
:102C3400D904226004D5421C01D12B6803B9606514
:102C4400616B2F600029CAD004F14403994202D079
:102C5400284600F09FF900206063BDE8F081216AF6
:102C640001232846B047411CC6D12B68002BC3D092
:102C74001D2B01D0162B01D12F60B0E7A38943F09F
:102C84004003A381BDE8F0810F69002FA7D093070B
:102C940018BF00230E6808BF4B69A6EB07080F6036
:102CA4008B60B8F1000F9ADD43463A46216A284604
:102CB400A66AB047002807DCA38943F04003A38138
:102CC4004FF0FF30BDE8F0810744A8EB0008E8E7C7
:102CD4000100402038B50B6905460C46DBB118B13C
:102CE40083690BB900F060F80C4B9C4209D16C6805
:102CF400B4F90C307BB121462846BDE83840FFF7D3
:102D040061BF074B9C4201D1AC68F1E7054B9C4283
:102D140008BFEC68ECE7002038BD00BFB8390008F4
:102D2400D839000898390008014900F0A9B800BF53
:102D3400D92C0008002310B5044603604360836067
:102D440081814366C281036143618361194608221C
:102D54005C30FFF73DFD054B24626362044BA362C4
:102D6400044BE362044B236310BD00BFB936000873
:102D7400DB360008133700083737000870B56825BC
:102D84004A1E55430E4605F1740100F04FF90446FE
:102D940040B1002180E842000C30A06005F16802D7
:102DA400FFF716FD204670BD836910B5044633BB9A
:102DB4008364C3640365124B124A1B68826298429F
:102DC40004BF0123836100F01FF86060204600F017
:102DD4001BF8A060204600F017F80022E0600421F0
:102DE4006068FFF7A7FF01220921A068FFF7A2FF8F
:102DF40002221221E068FFF79DFF0123A36110BDA9
:102E0400943900082D2D0008F8B51C4B07461E68A0
:102E1400B36913B93046FFF7C7FF4836B46873681F
:102E2400013B03D5336833B13668F7E7B4F90C5086
:102E34006DB16834F4E704213846FFF79FFF306032
:102E44000028F1D10C2304463B602046F8BD4FF620
:102E5400FF73E38101236566A3812560A560656036
:102E640025616561A5610822294604F15C00FFF72C
:102E7400AFFC6563A563A564E564E6E794390008DF
:102E84002DE9F84380468946002600F1480414B928
:102E94003046BDE8F883A5686768013F01D524681A
:102EA400F5E7AB89012B07D9B5F90E30013303D00F
:102EB40029464046C84706436835EEE770B50E46D6
:102EC400B1F90E1090B0002914461D4607DA00230C
:102ED4002B60B3891A0610D44FF480630EE001AA64
:102EE40000F04EFC0028F2DB029A02F47042A2F5D4
:102EF40000535A425A412A60EEE7402300202360DF
:102F040010B070BD8B8973B59D0706460C4607D576
:102F140004F14703236023610123636102B070BDA0
:102F240001AB6A46FFF7CAFF00990546304600F038
:102F34007DF848B9B4F90C309A05EFD423F00303B3
:102F440043F00203A381E3E70D4BB362A38920603E
:102F540043F08003A381009B20616361019B5BB10B
:102F6400B4F90E10304600F01DFC28B1A38923F0FB
:102F7400030343F00103A381A3891D43A581CDE786
:102F84002D2D0008024B0146186800F04FB800BF11
:102F94001C02002038B50546002943D051F8043CF2
:102FA4000C1F002BB8BFE41800F02CFC1E4A136859
:102FB400104633B9636014602846BDE8384000F019
:102FC40022BCA3420BD921686218934201BF1A683C
:102FD4005B685218226063600460EDE713465A6828
:102FE4000AB1A242FAD919685818A0420BD1206834
:102FF4000144581882421960DED1106852680144B5
:1030040019605A60D8E702D90C232B60D4E72068F2
:1030140021188A4201BF1168526809182160626050
:103024005C60C9E738BD00BFF002002070B5CD1C5C
:1030340025F0030508350C2D38BF0C25002D064658
:1030440001DBA94203D90C233360002070BD00F0DA
:10305400D9FB234A1468214691B9224C23681BB931
:10306400304600F017FB20602946304600F012FB82
:10307400431C26D10C233046336000F0C4FBE4E744
:103084000B685B1B1AD40B2B0FD90B60CC18CD50DB
:10309400304600F0B8FB04F10B00231D20F00700BC
:1030A400C31A1BD05A42E25070BD8C420BBF6368F6
:1030B4004B681360636018BF0C46E9E70C46496827
:1030C400CAE7C41C24F00304A04205D0211A3046E8
:1030D40000F0E0FA0130CDD02560D9E770BD00BF23
:1030E400F0020020F4020020936810B4013B002B8E
:1030F400936008DA9469A34202DBCBB20A2B02D1B3
:1031040010BCFFF79FBC1368581C10601970C8B23C
:1031140010BC7047F8B506460F461446D518AC42A5
:1031240001D1002007E03A4614F8011B3046FFF7AE
:10313400DBFF431CF3D1F8BD2DE9F04F9DB00C46E5
:1031440017460393064618B183690BB9FFF72CFEA3
:103154007C4B9C4257D17468A38918075DD52369B9
:10316400002B5AD00023099320238DF829303023D3
:103174004FF0010B8DF82A30B846454615F8013B4F
:10318400002B55D1B8EB070A0BD053463A462146DB
:103194003046FFF7BFFF013000F0C480099B534461
:1031A400099398F80030002B00F0BC8000234FF006
:1031B400FF3204930793059206938DF853301A93C4
:1031C40005222978604800F00FFB05F10108049BF3
:1031D400002831D1D90644BF20228DF853201A0784
:1031E40044BF2B228DF853202A782A2A2CD0002180
:1031F4000A20079AA84698F800300135303B092B7D
:103204006DD971B326E0514B9C4201D1B468A3E758
:103214004F4B9C4208BFF4689EE721463046FFF7B7
:1032240063FC00289ED04FF0FF301DB0BDE8F08F46
:10323400252BA7D0A846A0E7434A4546801A0BFA97
:1032440000F018430490BBE7039A111D1268039120
:10325400002A01DB079204E0524243F00203079282
:10326400049398F800302E2B10D198F8013008F10F
:1032740001012A2B37D1039B08F102081A1D1B6890
:103284000392002BB8BF4FF0FF330593314D032257
:1032940098F80010284600F0A7FA40B14023401BDC
:1032A40003FA00F0049B08F101080343049398F81F
:1032B40000100622284808F101078DF8281000F0B4
:1032C40093FA002834D0254B03BB039B073323F028
:1032D400070308330393099B4B4409934CE700FB12
:1032E4000232012186E700230A2518460593884601
:1032F40098F800200131303A092A03D9002BC5D0AF
:103304000590C3E705FB00200123F0E703AB00931E
:103314002246134B04A93046AFF30080B0F1FF3FBF
:103324008146D8D1A3895B063FF57DAF09987CE738
:1033340003AB009322460A4B04A9304600F08AF8F6
:10334400ECE700BFB8390008F8390008D83900089C
:1033540098390008FE390008023A0008000000000D
:10336400193100082DE9F04791461F468A680B6918
:1033740006469342B8BF1346C9F8003091F843207B
:103384000C46DDF8208012B10133C9F800302368FF
:10339400990642BFD9F800300233C9F800302568D5
:1033A40015F0060507D104F1190AE368D9F80020DD
:1033B4009B1A9D422ADB94F843302268003318BFDD
:1033C400012392062FD404F1430239463046C04704
:1033D400013022D02368E56803F00603042B18BFEC
:1033E4000025D9F800204FF0000908BFAD1AA368E2
:1033F400226908BF25EAE5759342C4BF9B1AED18FC
:103404001A344D451BD10020BDE8F08701235246F4
:1034140039463046C047013003D14FF0FF30BDE894
:10342400F0870135C1E73020E11881F843005A1CC8
:1034340094F845102244023382F84310C3E7012371
:10344400224639463046C0470130E6D009F1010929
:10345400D7E700002DE9F04317460A7E85B06E2AAF
:10346400984606460C460C9B01F1430E00F0BC80C6
:103474001AD8632A2ED00AD8002A00F0C880582A05
:1034840000F08A8004F1420584F842202AE0642A8C
:1034940001D0692AF6D121681A6811F0800F23D06F
:1034A400111D1960136827E0732A00F0B48008D84E
:1034B4006F2A2AD0702AE5D10A6842F020020A60F5
:1034C40003E0752A21D0782ADCD178226F4984F868
:1034D400452064E01A6801F14205111D1960136862
:1034E40084F842300123A3E011F0400F02F10401FB
:1034F4001960D7D0B2F90030002B03DA2D225B42D9
:1035040084F8432062490A2217E02068196810F001
:10351400800F03D0081D18600B6806E010F0400F00
:1035240001F104001860F7D00B886F2A14BF0A2237
:1035340008225749002084F843006568002DA560DF
:10354400C0F29C80206820F004002060002B3FD152
:10355400002D40F095807546082A0BD12368DA07C0
:1035640008D5236962689A42DEBF302305F8013C1E
:1035740005F1FF35AEEB05032361CDF800803B4632
:1035840003AA21463046FFF7EDFE013055D14FF036
:10359400FF3005B0BDE8F08381F845203C4922683E
:1035A400186812F0800F00F104051D6001D0036853
:1035B40002E05506FBD50388D00744BF42F0200241
:1035C40022601BB9226822F0200222601022B1E797
:1035D4007546B3FBF2F002FB1033CB5C05F8013DFA
:1035E40003460028F5D1B7E708681A6810F0800F81
:1035F400496904D0101D18601368196007E010F0C1
:10360400400F02F1040018601368F6D019800023FB
:1036140075462361B1E71A68111D19601568002108
:103624006268284600F0E0F808B1401B60606368F7
:103634002361002384F843309FE723692A463946EF
:103644003046C0470130A2D023689B0707D5002528
:1036540004F11909E368039A9B1A9D4205DBE068AB
:10366400039B9842B8BF184693E701234A4639465C
:103674003046C04701308AD00135EBE7002BA7D193
:103684000B7804F1420584F8423065E71A3A0008E1
:10369400093A000838B50023054C0546084623605E
:1036A400FEF75AFF431C02D1236803B12B6038BDD7
:1036B4000412002010B50C46B1F90E1000F0A4F865
:1036C4000028ABBF636DA3891B1823F48053ACBFE0
:1036D4006365A38110BD2DE9F0411F468B89054622
:1036E400DB050C46164605D502230022B1F90E105F
:1036F40000F068F8A389324623F48053A381B4F917
:103704000E103B462846BDE8F04100F017B810B54E
:103714000C46B1F90E1000F055F8431CA38915BFEF
:10372400606523F4805343F48053A38118BFA381BD
:1037340010BDB1F90E1000F013B8000038B50546FD
:10374400084611460022054C22601A46FEF776FC14
:10375400431C02D1236803B12B6038BD041200203E
:1037640038B50023054C054608462360FEF70EFFD6
:10377400431C02D1236803B12B6038BD041200201E
:1037840038B50023064C0546084611462360FEF76B
:1037940000FF431C02D1236803B12B6038BD00BF76
:1037A4000412002038B50023054C05460846236062
:1037B400FEF7F4FE431C02D1236803B12B6038BD2D
:1037C4000412002038B50546084611460022054C6F
:1037D40022601A46FEF7E4FE431C02D1236803B1BB
:1037E4002B6038BD0412002010B5C9B202449042C7
:1037F400034601D1002010BD1C7801308C42F6D163
:10380400184610BD7047704738B50546084611463E
:103814000022054C22601A46FEF790FE431C02D19A
:10382400236803B12B6038BD04120020F8B500BF33
:10383400F8BC08BC9E467047F8B500BFF8BC08BC8D
:043844009E467047E5
:1038480002030405060708090A0B0C0D0E0F1010D9
:10385800253032782000436865636B2053756D20EE
:103868006572726F72200075706461746520436FB1
:103878006D706C65746520004465766963652054D5
:103888006F74616C203A2025640D0A2020202020C6
:1038980046696C65202020546F74616C203A20259D
:1038A800640D0A2020202000446576696365205451
:1038B8006F74616C203A2025640D0A202020204670
:1038C800696C65202020546F74616C203A2025644F
:1038D8000D0A202020200048414C5F464C415348A7
:1038E8005F50726F6772616D2829206572726F72FE
:1038F800203078253038782C20736565202A686157
:103908006C5F666C6173682E6820666F72206269EE
:103918007420646566696E6974696F6E730A00481D
:10392800414C204E4F54204F4B2000457261736527
:10393800204661696C6564200D00626F6F74206CAD
:103948006F61646572207374617274006A756D705A
:103958002100000000000000000001020304060727
:1039680008090000000001020304435243204552A5
:1039780052202578200D0A00434845434B205355D3
:103988004D20455252202578200D0A0020020020A3
:10399800000000000000000000000000000000001F
:1039A800000000000000000000000000000000000F
:1039B80000000000000000000000000000000000FF
:1039C80000000000000000000000000000000000EF
:1039D80000000000000000000000000000000000DF
:1039E80000000000000000000000000000000000CF
:1039F800232D302B2000686C4C00656667454647D0
:103A08000030313233343536373839414243444552
:103A180046003031323334353637383961626364C1
:043A280065660000CF
:043A2C000902000883
:043A3000E5010008A4
:103A34000100000010000000BE11030500BEBE0B13
:103A4400030400EB00002110422063308440A550A1
:103A5400C660E770088129914AA16BB18CC1ADD1D0
:103A6400CEE1EFF13112100273325222B552944278
:103A7400F772D662399318837BB35AA3BDD39CC320
:103A8400FFF3DEE36224433420040114E664C774C4
:103A9400A44485546AA54BB528850995EEE5CFF570
:103AA400ACC58DD55336722611163006D776F66618
:103AB4009556B4465BB77AA719973887DFF7FEE7C0
:103AC4009DD7BCC7C448E5588668A77840086118E4
:103AD40002282338CCC9EDD98EE9AFF94889699910
:103AE4000AA92BB9F55AD44AB77A966A711A500AB8
:103AF400333A122AFDDBDCCBBFFB9EEB799B588B60
:103B04003BBB1AABA66C877CE44CC55C222C033C03
:103B1400600C411CAEED8FFDECCDCDDD2AAD0BBDAF
:103B2400688D499D977EB66ED55EF44E133E322E57
:103B3400511E700E9FFFBEEFDDDFFCCF1BBF3AAFFF
:103B4400599F788F8891A981CAB1EBA10CD12DC15D
:103B54004EF16FE18010A100C230E32004502540F3
:103B640046706760B9839893FBA3DAB33DC31CD353
:103B74007FE35EF3B1029012F322D2323542145243
:103B840077625672EAB5CBA5A89589856EF54FE59F
:103B94002CD50DC5E234C324A01481046674476493
:103BA40024540544DBA7FAB79987B8975FE77EF7F3
:103BB4001DC73CD7D326F2369106B01657667676E3
:103BC400154634564CD96DC90EF92FE9C899E989BF
:103BD4008AB9ABA94458654806782768C018E10833
:103BE4008238A3287DCB5CDB3FEB1EFBF98BD89B93
:103BF400BBAB9ABB754A545A376A167AF10AD01A83
:103C0400B32A923A2EFD0FED6CDD4DCDAABD8BADDE
:103C1400E89DC98D267C076C645C454CA23C832CD2
:103C2400E01CC10C1FEF3EFF5DCF7CDF9BAFBABF32
:103C3400D98FF89F176E367E554E745E932EB23E22
:103C4400D10EF01E0050000800A24A0420020020F9
:103C540000000000B8390008D83900089839000875
:103C64000000000000000000000000000000000050
:103C74000000000000000000000000000000000040
:103C84000000000000000000000000000000000030
:103C94000000000000000000000000000000000020
:103CA4000000000000000000000000000000000010
:040000050800273593
:00000001FF
